:100AB8001201000200000040051601800100010239
:100AC80000010A060002000000400100090220009F
:100AD800010100A0320904000002FF000000070520
:100AE8000202000200070586020002000902200037
:100AF800010100A0320904000002FF000000070500
:100B080001024000000705810240000004030904B7
:100B180026034100430043004500530020004900DC
:100B28002F004F002000500072006F006400750015
:100B380063007400730016035500530042002D0033
:0E0B4800440049004F002D0033003200000031
:03004300020A00AE
:03005300020A009E
:100A0000020EB600020F3B00020F2500020F0D0080
:100A1000020CFA00020D3100020032000200420016
:100A200002005200020F9F00020FA000020FA1005F
:100A3000020FA200020FA300020FA400020FA500E4
:100A4000020FA60002004200020FA700020FA8003A
:100A5000020FA900020FAA00020FAB00020FAC00A8
:100A6000020FAD00020042000200420002004200FC
:100A7000020FAE00020FAF00020FB000020FB10074
:100A8000020FB200020FB300020FB400020FB50054
:100A9000020FB600020FB700020FB800020FB90034
:100AA000020FBA00020FBB00020FBC00020FBD0014
:080AB000020FBE00020FBF009F
:0A09F40000010202030304040505DC
:10096300E4F50BF50AF509F508C203C200C202C299
:100973000112003675230A7524B8752B0A752CCA23
:1009830075210A7522D475290A752AF4752D0B75FC
:100993002E14D2E843D82090E668E04409F090E6AC
:1009A3005CE0443DF0D2AFD20412000390E680E055
:1009B30054F7F0538EF8C20330010512056DC201DE
:1009C3003003291209FE5024C203120E912000168F
:1009D30090E682E030E704E020E1EF90E682E03049
:1009E300E604E020E0E4120E39120F95120BE280C8
:0109F300C73C
:10056D0090E6B9E0700302061E14700302069B2488
:10057D00FE700302071E24FB70030206181470039D
:10058D000206121460731460762405600302077D61
:10059D00120F97400302078990E6BBE024FE60220C
:1005AD0014603324FD601114602224067048E52385
:1005BD0090E6B3F0E5248037E52B90E6B3F0E52C1B
:1005CD00802DE52590E6B3F0E5268023E52790E61E
:1005DD00B3F0E528801990E6BAE0FF120E65AA0681
:1005ED00A9077B01EA494B600DEE90E6B3F0EF9061
:1005FD00E6B4F0020789020782120F63020789121F
:10060D000F7D020789120F75020789120F5102071C
:10061D0089120F99400302078990E6B8E0247F60A4
:10062D001514601924027063A200E43325E0FFA2C3
:10063D0002E4334F8041E490E740F0803F90E6BC08
:10064D00E0547EFF7E00E0D394807C0040047D0169
:10065D0080027D00EC4EFEED4F24F4F58274093ED0
:10066D00F583E493FF3395E0FEEF24A1FFEE34E62E
:10067D008F82F583E0540190E740F0E4A3F090E61B
:10068D008AF090E68B7402F0020789020782120F3E
:10069D009B400302078990E6B8E024FE6016240211
:1006AD00600302078990E6BAE0B40105C2000207B3
:1006BD008902078290E6BAE0705590E6BCE0547E60
:1006CD00FF7E00E0D394807C0040047D0180027D9C
:1006DD0000EC4EFEED4F24F4F58274093EF583E4F3
:1006ED0093FF3395E0FEEF24A1FFEE34E68F82F504
:1006FD0083E054FEF090E6BCE05480131313541FB6
:10070D00FFE0540F2F90E683F0E04420F0806D80E1
:10071D0064120F9D506690E6B8E024FE6019240225
:10072D00705A90E6BAE0B40104D200804F90E6BA58
:10073D00E064026047803E90E6BCE0547EFF7E00A0
:10074D00E0D394807C0040047D0180027D00EC4E5E
:10075D00FEED4F24F4F58274093EF583E493FF33E7
:10076D0095E0FEEF24A1FFEE34E68F82F58380083D
:10077D00120056500790E6A0E04401F090E6A0E08C
:03078D004480F0B5
:010790002246
:0300330002004E7A
:04004E0053D8EF3262
:04004600022F000085
:0C003600D200120F85E4F5B175B63F2230
:040F8D0043B120222A
:040F910053B1DF2257
:100BE200E5336035E530452F7006752F2F7530FFE0
:100BF200E53015307002152FE530452F7004F533BE
:100C0200800FAE2FAF307C0B7DFF1208E8EF20E0A3
:100C120005120F918003120F8DE5B190E68020E757
:0A0C220005E04408F022E054F7F06A
:010C2C0022A5
:0209FE00D32202
:020F9500D32265
:020F9700D32263
:080F750090E6BAE0F534D32246
:100F510090E740E534F0E490E68AF090E68B04F007
:020F6100D32299
:080F7D0090E6BAE0F531D32241
:100F630090E740E531F0E490E68AF090E68B04F0F8
:020F7300D32287
:020F9900D32261
:020F9B00D3225F
:020F9D00D3225D
:1000560075330190E678E05410C4540F4450F532DD
:1000660013E433F53590E6B9E012093D023F070186
:100076005410016611018412025D200321210342FE
:1000860023056B28056B2C056B2D056B2E01FC30AB
:1000960001FC3103E7A203E7A303E1A903B7AC051B
:1000A6006BF000B5F100CBF2056BF300000569902B
:1000B600E6BAE0F580A3E0F590A3E0F5A0A3E0F5AD
:1000C600B0E402031A90E6BEE0750E00F50FA3E059
:1000D600FEEE420EE50F450E700490E68BF0E50F3E
:1000E600450E700302056B90E6A0E020E1F9C3E53A
:1000F6000F9440E50E94005008850E10850F118070
:1001060006751000751140E4F512F513C3E5139555
:1001160011E5129510501DAF13C3E50F9FFE7440F5
:100126002FF582E434E7F583EEF00513E51370DC72
:10013600051280D8E490E68AF090E68BE511F0C3CC
:10014600E50F9511F50FE50E9510F50E809090E6EA
:10015600BEE090E68BF090E6A0E020E1F90201E730
:1001660090E740E580F0A3E590F0A3E5A0F0A3E5D5
:10017600B0F0E490E68AF090E6BEE002031AE4905E
:10018600E68AF090E6BEE090E68BF090E6A0E020EE
:10019600E1F990E744E030E0047FFF80027F008FC2
:1001A600B290E744E030E1047FFF80027F008FB326
:1001B60090E744E030E2047FFF80027F008FB49036
:1001C600E744E030E3047FFF80027F008FB590E6CE
:1001D600BAE05401C454F0FF90E744E0540F4FF5E1
:1001E600B190E740E0F580A3E0F590A3E0F5A0A389
:1001F600E0F5B002056B90E740E580F0A3E590F0EE
:10020600A3E5A0F0A3E5B0F0E5B130E4047F0180FA
:10021600027F0090E6BAEFF0E5B1540F90E744F0A4
:10022600A37469F0A304F0A304F0A304F0E490E639
:100236008AF090E6BEE002031A90E6BAE0FF120EDC
:1002460065AA06A9077B01EA494B6009EE90E6B369
:10025600F0EF0203DAD32290E6BEE0B4022090E685
:10026600BBE0C4333354C0FF90E6BAE075F008A48F
:100276002403F582E5F03480F583EFF0805290E6B2
:10028600BEE06403704A90E6BBE0FF7401A807086D
:100296008002C333D8FC25E044C0FF90E6BAE0757F
:1002A600F008A42403F582E5F03480F583EFF0909E
:1002B600E6BAE075F008A4FFA3E07C002FFFEC355A
:1002C600F0FEE42FF58274803EF583E090E742F07D
:1002D60090E6BAE075F008A4FFA3E07C002FFFECDF
:1002E60035F0FEE42FF58274803EF583E090E7401A
:1002F600F090E6BAE075F008A4FFA3E02FFFEC3516
:10030600F0FEE42FF58274803EF583E090E741F03D
:1003160090E6BEE090E68BF002056BE490E68BF08B
:1003260090E6BBE0FF90E6BAE075F008A42403F57A
:1003360082E5F03480F583EFF002056BE490E68BFE
:10034600F090E6BBE0FF90E6BAE075F008A424035F
:10035600F582E5F03480F583EFF090E6BCE0FD90A1
:10036600E6BBE0C4131354037A005403FB90E6BAC9
:10037600E075F008A42BFFEA35F0FEE42FF5827451
:10038600803EF583EDF090E6BDE0FD90E6BBE0C46F
:1003960013135403FB90E6BAE075F008A42BFFEAAA
:1003A60035F0FEE42FF58274803EF583EDF002050C
:1003B6006B90E6B5E054FEF090E6BFE090E68AF07A
:1003C60090E6BEE090E68BF090E6BBE090E6B3F0F8
:1003D60090E6BAE090E6B4F002056B75350143325B
:1003E6000190E6BAE0750C00F50DA3E0FEEE420CB6
:1003F60090E6BEE0750E00F50FA3E0FEEE420E900D
:10040600E6B8E064C060030204D3E50F450E70034E
:1004160002056B90E6A0E020E1F9C3E50F9440E504
:100426000E94005008850E10850F11800675100079
:1004360075114090E6B9E0B4A335E4F512F513C39F
:10044600E5139511E5129510505EE50D2513F5821D
:10045600E50C3512F583E0FF74402513F582E4348C
:10046600E7F583EFF00513E51370D4051280D0E4A9
:10047600F512F513C3E5139511E51295105018748E
:10048600402513F582E434E7F58374CDF00513E5D2
:100496001370E1051280DDAD117AE779407F40AB3C
:1004A60007AF0DAE0C120C2DE490E68AF090E68BA9
:1004B600E511F0250DF50DE510350CF50CC3E50F2E
:1004C6009511F50FE50E9510F50E02041090E6B89D
:1004D600E06440600302056BE50F450E70030205FC
:1004E6006BE490E68AF090E68BF090E6A0E020E1DF
:1004F600F990E68BE0751000F51190E6B9E0B4A32B
:1005060035E4F512F513C3E5139511E51295105070
:100516003674402513F582E434E7F583E0FFE50DF4
:100526002513F582E50C3512F583EFF00513E51377
:1005360070D4051280D0AD117AE779407F40AB07C1
:10054600AF0DAE0C120D9EE511250DF50DE510351E
:100556000CF50CC3E50F9511F50FE50E9510F50E8C
:060566000204DED322C3F3
:01056C00226C
:100EB600C0E0C083C08290E6B5E04401F0D20153A1
:0F0EC60091EF90E65D7401F0D082D083D0E032DE
:100F2500C0E0C083C0825391EF90E65D7404F0D0B9
:060F350082D083D0E032FF
:100F3B00C0E0C083C0825391EF90E65D7402F0D0A5
:060F4B0082D083D0E032E9
:100CFA00C0E0C083C08290E680E030E70E852125FF
:100D0A00852226852927852A28800C852925852A52
:100D1A00268521278522285391EF90E65D7410F0ED
:070D2A00D082D083D0E0323B
:100F0D00C0E0C083C082D2035391EF90E65D7408B8
:080F1D00F0D082D083D0E03255
:100D3100C0E0C083C08290E680E030E70E852125C7
:100D4100852226852927852A28800C852925852A1B
:100D5100268521278522285391EF90E65D7420F0A6
:070D6100D082D083D0E03204
:01003200329B
:01004200328B
:01005200327B
:010F9F00321F
:010FA000321E
:010FA100321D
:010FA200321C
:010FA300321B
:010FA400321A
:010FA5003219
:010FA6003218
:010FA7003217
:010FA8003216
:010FA9003215
:010FAA003214
:010FAB003213
:010FAC003212
:010FAD003211
:010FAE003210
:010FAF00320F
:010FB000320E
:010FB100320D
:010FB200320C
:010FB300320B
:010FB400320A
:010FB5003209
:010FB6003208
:010FB7003207
:010FB8003206
:010FB9003205
:010FBA003204
:010FBB003203
:010FBC003202
:010FBD003201
:010FBE003200
:010FBF0032FF
:040CBB00AA06AC05D4
:100CBF00E4FD7E000DEE2400F582E43400F583EAB6
:100CCF00F00E0D74002EF582E43400F583EFF00D75
:100CDF0074002402F582E43400F583ECF07A007B93
:0B0CEF0000AF32120EF1AF32020D68B0
:0A0D9E008E148F158D168A178B181E
:100DA800E4F519E519C3951650200515E515AE1497
:100DB8007002051414FFE5182519F582E43517F5B6
:0A0DC80083E0FD120CBB051980D971
:010DD20022FE
:0A0C2D008E148F158D168A178B1890
:100C3700E4FDF519E5356012E514FF7E000DEE249D
:100C470000F582E43400F583EFF0AE050D74002E55
:100C5700F582E43400F583E515F07A007B00AF32C6
:0E0C6700120EF1AB18AA17AD16AF32020ED561
:100E390090E682E030E004E020E60B90E682E030C4
:100E4900E119E030E71590E680E04401F07F147E77
:0C0E590000120C7590E680E054FEF022C0
:100E910090E682E044C0F090E681F04387010000D3
:040EA100000000222B
:1000030030040990E680E0440AF0800790E680E03F
:100013004408F07FDC7E05120C7590E65D74FFF0FA
:0F00230090E65FF05391EF90E680E054F7F02203
:080F8500E4F51FD2E9D2AF220E
:100D680090E678E020E6F9C2E990E678E04480F081
:100D7800EF25E090E679F090E678E030E0F990E64B
:100D880078E04440F090E678E020E6F990E678E0F4
:060D980030E1D6D2E92291
:100E0700A90790E678E020E6F9E51F702390E678D9
:100E1700E04480F0E925E090E679F08D1AAF03A968
:100E270007751B018A1C891DE4F51E751F01D32256
:020E3700C322D4
:100DD300A90790E678E020E6F9E51F702590E6780C
:100DE300E04480F0E925E0440190E679F08D1AAF04
:100DF30003A907751B018A1C891DE4F51E751F03D2
:040E0300D322C32211
:03004B0002079118
:10079100C0E0C083C082C085C084C086758600C0A9
:1007A100D075D000C000C001C002C003C006C007A0
:1007B10090E678E030E206751F0602087B90E67845
:1007C100E020E10CE51F64026006751F0702087B4B
:1007D100E51F24FE605F14603624FE700302086C7E
:1007E10024FC70030208782408600302087BAB1B19
:1007F100AA1CA91DAF1E051E8F82758300120899C0
:1008010090E679F0E51E651A7070751F05806B9092
:10081100E679E0AB1BAA1CA91DAE1E8E8275830072
:100821001208C6751F02E51A6401704E90E678E061
:100831004420F08045E51A24FEB51E0790E678E0D5
:100841004420F0E51A14B51E0A90E678E04440F021
:10085100751F0090E679E0AB1BAA1CA91DAE1E8E88
:10086100827583001208C6051E800F90E678E04469
:1008710040F0751F008003751F005391DFD007D032
:1008810006D003D002D001D000D0D0D086D084D001
:0808910085D082D083D0E03253
:020E6500A907DB
:100E6700AE2DAF2E8F828E83A3E064037017AD0182
:100E770019ED7001228F828E83E07C002FFDEC3EFE
:090E8700FEAF0580DF7E007F0054
:010E9000223F
:100ED500120DD3E51F24FA600E146006240770F383
:0C0EE500D322E4F51FD322E4F51FD32232
:100EF100120E07E51F24FA600E146006240770F332
:0C0F0100D322E4F51FD322E4F51FD32215
:100C75008E0C8F0D90E600E054187012E50D2401DE
:100C8500FFE4350CC313F50CEF13F50D801590E655
:100C950000E05418FFBF100BE50D25E0F50DE50C40
:100CA50033F50CE50D150DAE0C7002150C4E6005F7
:060CB500120EA580EE22E4
:100EA5007400F58690FDA57C05A3E582458370F960
:010EB500221A
:03000000020B569A
:0C0B5600787FE4F6D8FD758135020B9D18
:10089900BB010CE58229F582E5833AF583E0225014
:1008A90006E92582F8E622BBFE06E92582F8E2225E
:0D08B900E58229F582E5833AF583E4932278
:1008C600F8BB010DE58229F582E5833AF583E8F068
:1008D600225006E92582C8F622BBFE05E92582C814
:0208E600F222FC
:1008E800BC000BBE0029EF8DF084FFADF022E4CCF4
:1008F800F875F008EF2FFFEE33FEEC33FCEE9DECBD
:10090800984005FCEE9DFE0FD5F0E9E4CEFD22ED02
:10091800F8F5F0EE8420D21CFEADF075F008EF2F4C
:10092800FFED33FD4007985006D5F0F222C398FD3D
:050938000FD5F0EA22DA
:10093D00D083D082F8E4937012740193700DA3A349
:10094D0093F8740193F5828883E47374029368605D
:06095D00EFA3A3A380DF5D
:100B6200020963E493A3F8E493A34003F68001F23D
:100B720008DFF48029E493A3F85407240CC8C33394
:100B8200C4540F4420C8834004F456800146F6DF63
:100B9200E4800B0102040810204080900046E47EAD
:100BA200019360BCA3FF543F30E509541FFEE49358
:100BB200A360010ECF54C025E060A840B8E493A31F
:100BC200FAE493A3F8E493A3C8C582C8CAC583CA4A
:100BD200F0A3C8C582C8CAC583CADFE9DEE780BE02
:01004A0000B5
:00000001FF
